:0300000002036098
:03004300020100B7
:1001000002013C000201580002011800020129000E
:10011000020120000201180032E591C2E4F59122AB
:10012000C0E0C2003119D0E032C0E0E5874401F5FB
:10013000870000003119D0E032C2DC32C0D0C0E00C
:10014000C082C08312016931197401907FABF0D075
:1001500083D082D0E0D0D032C0D0C0E0C082C08393
:090160001203DC3119740280E283
:10016900907FE8E0A2E79202545C7051E0A2E0823D
:10017900E1404A30E50274035403C4F540A3E05456
:100189000F45401201D52001343002182003209078
:100199007F027846754003E6F0158218D540F8E6E7
:1001A900907FB5F0754002907FB4E04540F022851C
:1001B9008240E583907FD4F0E540A380E675400353
:1001C90080E5E02582F58250020583229001FA310B
:1001D900CCE09001FA31CCC082C0837845E4F618AE
:1001E900F6187601907FEAE0F5F0A3E0C201C203B8
:1001F900226D404040404081406A74404040404048
:1002090040714040404040A540404040404040404F
:1002190040714240404040404040404040404040A2
:1002290040405663404040404040435D404040406C
:1002390040D201223000FA907FC5F0907FAAE054A5
:100249000160FBF00203B33000E7087618223000A2
:10025900E0F541223000DA08A641223000D50876BF
:100269000122760222E5F060061470C5D20022C28E
:100279000022D203149002C560B9149002D760B36A
:100289001470AE900318E5F0601EF54031CBE060C4
:10029900A0E5401480F2D203C394219002E960934F
:1002A900149002F9608D8089E0FFF5F07800F2087A
:0C02B900A3E0DFFAD0E0D0E0E5F021A9DE
:1002C500120101010000004042420001000101024B
:1002D5000001090222000101008032090400000129
:1002E50003000000092100010001221F000705810C
:1002F500034000640600FF0901A101190129021547
:100305000026FF0075089501810219012902950251
:100315009102C0040309042C035500530042002038
:1003250000440065007300690067006E002000420C
:1003350000790020004500780061006D0070006CB8
:100345000065001603490032004300200042007298
:1003550000690064006700650000007581EB759217
:100365007F78D6E254F3F2120391E24406F2E4F503
:100375002078ACF208F2087403F2087401F278AA46
:1003850074FFF275E80175A8C00080FD75406490A2
:10039500FB50A3E582458370F9D540F322E220E6C0
:1003A500FC2271A27480F2E0F3E230E0FC2278A531
:1003B50079A6907EC071A7E020E007A371AC7440D8
:1003C500F2227420F2E371AE7440F2E3907E80F085
:0803D500907FB77401F02222B1
:00000001FF
